:100000000C945001FFFFFFFF0C943406FFFFFFFF2D
:10001000FFFFFFFFFFFFFFFFFFFFFFFFFFFFFFFFF0
:10002000FFFFFFFFFFFFFFFFFFFFFFFFFFFFFFFFE0
:10003000FFFFFFFFFFFFFFFFFFFFFFFFFFFFFFFFD0
:10004000FFFFFFFF0C94AA05FFFFFFFF0C947C1B32
:100050000C94101CFFFFFFFFFFFFFFFFFFFFFFFFE0
:10006000FFFFFFFFFFFFFFFFFFFFFFFFFFFFFFFFA0
:100070004D6F6465202020202020202044656D6F76
:100080004D6F6465202020205374616E6420427996
:100090004D6F646520496E74657272757074656425
:1000A0000000000000000000000000000000000050
:1000B0004D6F64652020502D4C696D6974696E67C1
:1000C0000000000000000000000000000000000030
:1000D0000000000000000000000000000000000020
:1000E0000000000000000000000000000000000010
:1000F0004D6F6465202020204D61782E502E502EAB
:10010000202020424954204661696C757265202088
:10011000202047726F756E64204661756C742020D4
:100120002020505631204F76657220566F6C742017
:100130002020505632204F76657220566F6C742006
:1001400020202053797374656D2045727220202021
:100150002020525844204661696C75726520202029
:1001600020205056204F76657220506F77657220A0
:10017000204772696420566F6C74204572726F72EA
:1001800020477269642046726571204572726F72F1
:10019000202054565331204661696C7572652020C9
:1001A000202054565332204661696C7572652020B8
:1001B0002020545653204661696C757265202020BA
:1001C000202020202020202020202020202020202F
:1001D0000020506C6561736520576169742E2E2E66
:1001E00020002020204165726F2D536861727020BD
:1001F00020200042617474657279204661696C75D3
:1002000072652100496E7465726E616C20546D7068
:100210002020204300542D546F74616C2020202036
:1002200020202E206800542D546F646179202020F6
:100230002020202E206800452D546F74616C2020F2
:10024000202020206B576800452D546F6461792071
:100250002020202E206B57680056707632202020F8
:10026000202020202020202056005670763120208B
:100270002020202020202020205600506F75742040
:10028000202020202020202020205700566772693F
:10029000642020202020202020202056000001FF64
:1002A000CFEFD4E0CDBFDEBFCE51D0400AEA088305
:1002B0000024EFE2F3E014E0E036F10711F00192E0
:1002C000FBCF0083E0E7F0E0A0E0B1E012E000E067
:1002D0000BBFEF39F10721F0C89531960D92F9CF98
:1002E0000E946C07FFCFBC9AC498B99AC19A0000CB
:1002F0000000B89AC09A000000000000000022240C
:100300002ABA0000000009B303C00000000009B3CE
:1003100007FDFBCFC0988FEF8ABB08958FEF8ABB94
:10032000BC9AC498B99AC198000000000BBB0000A9
:100330000000B89AC09A0000000000000000C098B9
:1003400008958FEF8ABBBC9AC49AB99AC1980000ED
:1003500000000BBB00000000B89AC09A000000002B
:1003600000000000C098089508E3D8DF08EC10E012
:100370000E94661B08E3D2DF08EC10E00E94661BB7
:1003800008E3CCDF08EC10E00E94661BACDF08E35A
:10039000C5DFA9DF08E0C2DFA6DF01E0BFDFA3DF22
:1003A00006E0BCDFA0DF0FE0B9DF9DCF0E946C1F2D
:1003B0005901C02ECC2019F402E0B0DF02C000ECDD
:1003C000ADDF91DF442706C0F50101915F01B9DF80
:1003D0008ADF43954031C0F30C94731F0E94541F71
:1003E000A901B80128EE33E08B010E94941EC801D8
:1003F000C096FA01838728EE33E08B010E94921E9B
:10040000B80124E630E00E94941EC801C096FA01AB
:10041000848724E630E08B010E94921EB8012AE016
:1004200030E00E94941EC801C096FA0185872AE038
:1004300030E08B010E94921EB801CB01C096FA01F8
:1004400086870C94591F0E94681E4A935A934E81C6
:100450005F8180E492E4AFE0B0E00A811B812C81EF
:100460003D81BA93AA939A938A930E94B01E0A83FD
:100470001B832C833D8380EA96E8A1E0B0E00A81EB
:100480001B812C813D81BA93AA939A938A930E94EF
:10049000AE1E1801290180E390E0A0E0B0E0280E34
:1004A000391E4A1E5B1EFA013996208280EA96E8C0
:1004B000A1E0B0E00A811B812C813D81BA93AA930F
:1004C0009A938A930E94B01E0A831B832C833D83D8
:1004D00080E197E2A0E0B0E00A811B812C813D81A0
:1004E000BA93AA939A938A930E94AE1E1801290187
:1004F00080E390E0A0E0B0E0280E391E4A1E5B1EAB
:10050000FA013A96208280E197E2A0E0B0E00A8109
:100510001B812C813D81BA93AA939A938A930E945E
:10052000B01E0A831B832C833D8388EE93E0A0E0FA
:10053000B0E00A811B812C813D81BA93AA939A93E2
:100540008A930E94AE1E1801290180E390E0A0E08A
:10055000B0E0280E391E4A1E5B1EFA013B9620822F
:1005600088EE93E0A0E0B0E00A811B812C813D8100
:10057000BA93AA939A938A930E94B01E0A831B830C
:100580002C833D8384E690E0A0E0B0E00A811B81EB
:100590002C813D81BA93AA939A938A930E94AE1EAE
:1005A0001801290180E390E0A0E0B0E0280E391E98
:1005B0004A1E5B1EFA013C96208284E690E0A0E091
:1005C000B0E00A811B812C813D81BA93AA939A9352
:1005D0008A930E94B01E0A831B832C833D838AE08A
:1005E00090E0A0E0B0E00A811B812C813D81BA93AC
:1005F000AA939A938A930E94AE1E1801290180E360
:1006000090E0A0E0B0E0280E391E4A1E5B1EFA0101
:100610003D9620828AE090E0A0E0B0E00A811B8154
:100620002C813D81BA93AA939A938A930E94B01E1B
:100630000A831B832C833D8380E390E0A0E0B0E03D
:100640002A803B804C805D80280E391E4A1E5B1E2E
:10065000FA01268659914991249608954A935A930E
:10066000402F4F7089E0841710F4495C01C0405D51
:10067000042F5991499108954A935A93402F552731
:100680005595479555954795559547955595479552
:1006900089E0841710F4495C01C0405D042F599132
:1006A000499108954A9344270BC0E42FFF27E20F96
:1006B000F31F2080E42FFF27E00FF11F20824395D6
:1006C000403198F3499108954A93442712C080E13C
:1006D000829F100180E091E0280E391EE42FFF2751
:1006E000E20DF31D2080E42FFF27E00FF11F208291
:1006F0004395403160F349910895AA92A02E6097E6
:100700002CE133E08E01CEDF9E018AE090E0009183
:10071000CF031091D0032F933F939C010E94941E0E
:100720003F912F915BDE8B85803339F480E28B879C
:100730008C85803311F480E28C879E010A2D36DE91
:100740006096A9900895AA92A02E60972BE033E0BE
:100750008E01A8DF9E010091BD031091BE033EDE15
:100760008B85803361F480E28B878C85803339F40C
:1007700080E28C878D85803311F480E28D879E0125
:100780000A2D14DE6096A9900895AA92A02E609773
:100790002AEF32E08E0186DF9E018AE090E0009130
:1007A000C9031091CA032F933F939C010E94941E8A
:1007B0003F912F9113DE8B85803339F480E28B8754
:1007C0008C85803311F480E28C879E010A2DEEDD4A
:1007D0006096A9900895AA92A02E609729EE32E023
:1007E0008E0160DF9E018AE090E00091C7031091C6
:1007F000C8032F933F939C010E94941E3F912F9119
:10080000EDDD8B85803339F480E28B878C858033F6
:1008100011F480E28C879E010A2DC8DD6096A990B4
:100820000895AA92A02E609728ED32E08E013ADF5B
:100830009E010091A4031091A503D0DD2C8429868C
:100840002D842A862E842C868EE28B878BE68D87DC
:1008500087E58E878985803311F480E289879E0140
:100860000A2DA4DD6096A9900895AA92A02E629701
:1008700027EC32E08E010E5F1F4F14DFCE0102968F
:10088000998388832091B1033091B2030091AF0323
:100890001091B003D8DD2B8429862C842A862D84E0
:1008A0002B862E842C862F842D8628882E868BE6F8
:1008B0008F8787E5888B89858033B1F480E28987CB
:1008C0008A85803389F480E28A878B85803361F45E
:1008D00080E28B878C85803339F480E28C878D852C
:1008E000803311F480E28D879E012E5F3F4F0A2DE9
:1008F0005DDD6296A9900895AA92A02E609726EBDE
:1009000032E08E01CFDE9E010091A7031091A80373
:1009100065DD8B85803339F480E28B878C8580336D
:1009200011F480E28C872B842A862C842B862D84DC
:100930002C868EE28D879E010A2D38DD6096A99067
:100940000895AA92A02E629725EA32E08E010E5FEA
:100950001F4FA8DECE010296998388832091AC03B5
:100960003091AD030091AA031091AB036CDD8B8530
:10097000803389F480E28B878C85803361F480E258
:100980008C878D85803339F480E28D878E85803326
:1009900011F480E28E872B842A862C842B862D846A
:1009A0002C862E842D862F842E868EE28F879E01A4
:1009B0002E5F3F4F0A2DFADC6296A9900895AA9205
:1009C0004A93A02E609744278091B7039091B80373
:1009D0008030E0E89E0738F0805090489093B8034C
:1009E0008093B7034AEA24E932E08E015BDE9E0180
:1009F0008AE090E00091B7031091B8032F933F93E2
:100A00009C010E94941E3F912F91E8DC80E78B8728
:100A10008C85803311F480E28C874A3A11F48DE2A0
:100A20008C879E010A2DC2DC60964991A990089599
:100A3000AA92CA92A02E60978091B5039091B603B6
:100A40008F709070C82EC0921404282F8E013CDE47
:100A50009E010A2DABDC6096C990A9900895AA92D8
:100A60004A93A02E6097442713C080E18A9D10010D
:100A700080E991E0280E391EE42FFF27E20DF31DD7
:100A80002080CE01E42FFF27E80FF91F2082439535
:100A9000403158F39E01002789DC442708C0CE016D
:100AA000E42FFF27E80FF91F80E280834395403150
:100AB000B0F39E0101E07ADC60964991A990089517
:100AC000AA924A93A02E6097442713C080E18A9D82
:100AD000100180EF91E0280E391EE42FFF27E20D70
:100AE000F31D2080CE01E42FFF27E80FF91F20829D
:100AF0004395403158F39E01002758DC6096499198
:100B0000A9900895609723E832E08E01CBDD9E0125
:100B100000274CDC60960895609722E732E08E0152
:100B2000C1DD9E01002742DC21E632E08E01BADD04
:100B30009E0101E03BDC60960895AA92A02E60978A
:100B400020E532E08E01AEDD9E010A2D2FDC60969D
:100B5000A99008952A923A928A939A93AA93EA9333
:100B60002FB62A9286EC82BF80915C0490915D043E
:100B7000019690935D0480935C04883EE3E09E07B9
:100B8000C9F52224332430925D0420925C048091C4
:100B90005F048F5F80935F04809130048F5F809348
:100BA000300480915F04853038F020925F0480919A
:100BB000380381608093380320902E04222029F08E
:100BC000822D815080932E0408C08B988AB780684C
:100BD0008ABF8BB780688BBF939A20903304222002
:100BE00021F0822D815080933304809137038160FE
:100BF0008093370320903204222039F0822D8233F3
:100C000020F48F5F809332040FC0809132048233CE
:100C100059F480913803877F8093380384608093F0
:100C2000380322242092320420903104222039F00B
:100C3000822D823320F48F5F809331040CC0809129
:100C40003104823341F4809137038061809337030C
:100C500022242092310429902FBEE991A9919991E3
:100C600089913990299018958A938FB78A938BB779
:100C70008F778BBF8AB780688ABF8B9A93988EE1F3
:100C800080932E0489918FBF8991189586EC82BF3D
:100C900084E083BF89B7826089BF89B78E7F89BFAF
:100CA00008958FEF8ABB8BBB87BB88BB84BB85BB9A
:100CB00081BB82BB86B987B9089522972090A00393
:100CC0003090A1033092340320923303209021040A
:100CD000222061F42090250480E3829DC001C0970A
:100CE0008E96909313048093120412C020902504D2
:100CF00080E3829DC001C097E0912104FF273197D6
:100D0000EE0FFF1F8E0F9F1F90931304809312040A
:100D10000E945B1D209033032092E0032090340357
:100D20002092E1032090120430901304398228822B
:100D300020EE33E002E00E945C1D22960895229787
:100D40000E945B1D80912504992780509A4F01973E
:100D500090931304809312042AE030E00091A403DE
:100D60001091A5030E94941E0093E00320901204AA
:100D7000309013043982288220EE33E001E00E9493
:100D80005C1D229608951A930A93229740909E0321
:100D900050909F0320909C0330909D03309230032D
:100DA00020922F0350923203409231032092E003AD
:100DB000209030032092E103209031032092E2033F
:100DC000209032032092E303809127049927019712
:100DD000880F991F880F991F8057994F909313047C
:100DE000809312040E945B1D209012043090130423
:100DF0003982288220EE33E004E00E945C1D2496B4
:100E00000895AA92BA92A02E2A2D332735952795B8
:100E10003595279535952795359527950AE010E066
:100E20000E94301F8A2D99278F7090705C01A00E50
:100E3000B11E0A2DB990A990089500270BC0222752
:100E4000332703C000002F5F3F4F2F3FEFEF3E07D8
:100E5000C8F303950F3198F30895B8980000000087
:100E600000000000B09904C00AE010E00E94661B78
:100E70000000000000000000B89AC098089585E4C2
:100E800093E0E0914403FF27E80FF91F222420821A
:100E900004E014C085E493E0209044033324280E3A
:100EA000391E210181E493E0E02FFF27E80FF91FAD
:100EB0002080F2013080320C30820395809144030F
:100EC0008C5F081738F385E493E0E0914403FF2733
:100ED000E80FF91F008108952297F894E2DEB89890
:100EE000000000000000000011C00AE010E00E94B5
:100EF000661B86B38170813049F40AE010E00E94DD
:100F0000661B86B38170813009F401C0EECF00000A
:100F1000000000000000B89AC098A8988EDF0E94D8
:100F2000B4010E948C0589DF0E94B81C0E94A41C99
:100F30008C988D98949A959A00000000849946C0E8
:100F4000859944C004E610E00E94661B84993EC067
:100F500085993CC022242092140412C00E945B1D7B
:100F60002090140482E3829D1982088220EE33E0EF
:100F700002E30E945C1D809114048F5F809314042F
:100F8000809114048E3950F30E945B1D8DED9EE11B
:100F90009983888320EE33E003E20E945C1D80EE9B
:100FA00099E09093340380933303282E2092E0033A
:100FB000292E2092E1030E945B1D87EF95E0998323
:100FC000888320EE33E002E00E945C1D8C9A8D9AAB
:100FD000949A959A5BDE2DE000E01FE10E94DF1DF0
:100FE000319A0E94731C2090E90320922A0425DF85
:100FF000399A0E94041C8B98939A85B78C6085BFA0
:101000008BB780688BBF8AB780688ABFD8C026E15B
:1010100000EE15E00E94DF1D2090E00320922F03D8
:101020002090E103209230032090E20320923103CC
:101030002090E3032092320340903103509032031A
:1010400020902F03309030033092B0032092AF03F2
:101050005092B2034092B1032090E4032092AE0379
:101060002090E50320922F032090E6032092300386
:101070002090E703209231032090E803209232036E
:10108000409031035090320320902F033090300372
:101090003092AB032092AA035092AD034092AC036E
:1010A0002090E903209233032090EA032092340336
:1010B00020903303309034033092A8032092A7038A
:1010C0002090EB03209233032090EC032092340312
:1010D00020903303309034033092A5032092A40370
:1010E0002090ED03209233032090EE0320923403EE
:1010F00020903303309034033092A3032092A20354
:101100002090EF03209233032090F00320923403C9
:1011100020903303309034033092A1032092A00337
:101120002090F1032092A9032090F20320922F0334
:101130002090F303209230032090F4032092310397
:101140002090F503209232034090310350903203F7
:1011500020902F033090300330929D0320929C0307
:1011600050929F0340929E0326E100EE15E00E94FC
:10117000DF1D2090E00320922F032090E1032092B6
:1011800030032090E203209231032090E303209269
:101190003203409031035090320320902F0330905F
:1011A00030038090B1039090B2036090AF037090D1
:1011B000B003621473048404950409F401C027CFBA
:1011C00022242092D50327E002E00E94261E2090D0
:1011D00017042092220420901804209220042090CA
:1011E00019042092230420901B04209226042090AE
:1011F0001C042092280420901D0420922904809130
:1012000022048036C8F4809120048036A8F48091AE
:101210002304843288F43090260481E3831560F03F
:101220005090280482E1851538F089E9821520F074
:10123000332011F05520D9F422242092170481E0A4
:101240008093180484E08093190485E080931A0445
:1012500081E080931B0480E180931C0480931D0433
:1012600027E002E00E94B01D81E08093D5038091C9
:10127000D503813081F4809136038F7780933603D4
:10128000222433243092A5032092A4033092A80391
:101290002092A703F4C221E009E00E94261E2090BC
:1012A000170425FE28C021E00AE11FE10E94DF1D8E
:1012B0002090E0032092140483E0821530F48091A2
:1012C0003603806880933603DAC2809136038F77C5
:1012D00080933603809114048F5F8093E0030E9413
:1012E0005B1D8AE19FE19983888320EE33E001E072
:1012F0000E945C1DC4C222242092E0030E945B1D58
:101300008AE19FE19983888320EE33E001E00E9427
:101310005C1D809136038F778093360322242092C0
:10132000160426E0002711270E94DF1D2090E0030D
:10133000209220042090E103209223042090E303D4
:10134000209226042090E403209228042090E503B4
:10135000209229040091200454DDA02EA0921F04A5
:10136000009123044EDDA02EA092210400912604BA
:1013700048DDA02EA09225040091280442DDA02E75
:10138000A092270426E003E00E94261E0091170485
:1013900038DDA02EA09217040091180432DDA02E93
:1013A000A092180400911A042CDDA02EA0921A0419
:1013B00000911B0426DDA02EA0921B043090270470
:1013C000301609F477C0032DDEDC80E080939C03A7
:1013D00080939D0380939E0380939F032090270416
:1013E000332440901B0455242414350474F5342C04
:1013F000321881E0831530F02090250430901A04D3
:10140000321418F080E280931604809127048F5FD5
:101410008093270481E0809314040DC00091270479
:10142000B2DC809127048F5F80932704809114049D
:101430008F5F8093140420902704332440901B0472
:1014400055242414350454F335C0209027043090DB
:101450001B04321478F5822D8C3019F0832D8130E5
:1014600031F42090250430901A04321460F080E2A8
:101470008093160408C00091270485DC809127041E
:101480008F5F809327048CE020902704821598F7C3
:1014900081E08093270408C00091270474DC8091C8
:1014A00027048F5F8093270420901B04309027042B
:1014B000321490F300912804A4DCA02EA0922704FB
:1014C00020901A0430902504321409F43FC037DC10
:1014D000222433243092A5032092A4033092A8033F
:1014E0002092A703809125048F5F8093250420908C
:1014F0001B04309027043214A1F406C020DC809134
:1015000025048F5F809325042090250430901A04D1
:101510003214A0F71BC013DC809125048F5F8093E9
:1015200025048FE1209025048215A8F781E080939F
:10153000250406C004DC809125048F5F8093250478
:1015400020901A04309025043214A0F321E006EF15
:1015500015E00E94DF1D2090E0032092110484EB2F
:10156000821510F48093110480E08093B903809376
:10157000BA038093BB038093BC03222420921404FB
:1015800034C022E0A09014042A2C3324022D112709
:101590000050194F020D131D0E94DF1D2090E00323
:1015A000209233032090E1032092340320903303F0
:1015B00030903403442455248090BB039090BC03A6
:1015C0006090B9037090BA03620C731C841C951C64
:1015D0007092BA036092B9039092BC038092BB03ED
:1015E000809114048F5F8093140420901104309034
:1015F0001404321430F244EB50E060E070E02091CB
:10160000BB033091BC030091B9031091BA037A93E4
:101610006A935A934A930E94AE1E1093BE0300939E
:10162000BD0300912604EDDBA02EA092250420909E
:101630001A040215B1F520901B04309027043214CF
:1016400081F520901804309021043214D9F0832DB4
:101650008F5F8093210431DB222433243092A10355
:101660002092A00306C0809121048F5F8093210403
:1016700024DB2090210433244090180455242414A2
:1016800035048CF32090BD033090BE034090A2033C
:101690005090A303420C531C5092A3034092A20308
:1016A000ADC080911604803208F0A8C0809121045A
:1016B000873120F022242092210405C0809121044A
:1016C0008F5F80932104F9DA222433243092A1031E
:1016D0002092A003809121048F5F80932104309297
:1016E000A3032092A20328EE33E00091BD031091E2
:1016F000BE030E94941E2090AE033324200E311EA0
:101700002092AE0306C0D9DA809121048F5F8093C6
:10171000210487E1209021048215A8F72224209239
:101720002104CBDA2090250430901A04321408F0FA
:1017300049C0822D8F5F8093250413C022242092FC
:10174000210406C0BADA809121048F5F80932104BE
:10175000809121048831B0F3809125048F5F8093BC
:1017600025048FE120902504821540F781E08093C5
:10177000250413C022242092210406C09EDA809101
:1017800021048F5F80932104809121048831B0F37C
:10179000809125048F5F8093250420901A04309057
:1017A0002504321438F31CC022242092210406C0E0
:1017B00084DA809121048F5F809321048091210439
:1017C0008831B0F3809125048F5FA82EA092250464
:1017D000282E332440901A0455242414350424F36D
:1017E00022242092210406C068DA809121048F5FB0
:1017F00080932104809121048831B0F380911604F4
:10180000803208F43CC0222433243092A103209279
:10181000A0033092A5032092A4033092A803209243
:10182000A7032092160481E08093250414C022248B
:101830002092210406C041DA809121048F5F8093B9
:10184000210487E1209021048215A8F780912504C6
:101850008F5F809325048FE120902504821538F74F
:1018600081E08093250406C06ADA809125048F5FA9
:10187000809325048FE1209025048215A8F72090FD
:10188000A7033090A8032220F1F43320E1F4209044
:10189000A4033090A5032220B1F43320A1F4222424
:1018A0002092E0032092E1032092E2032092E303DE
:1018B0000E945B1D89EE95E09983888320EE33E0DA
:1018C00004E00E945C1D22242092A603332430925F
:1018D000BE032092BD0316E000911F040E94181F52
:1018E0008EE1809F0092E0030E945B1D86EF95E0F1
:1018F0009983888320EE33E001E00E945C1D22245E
:10190000209214041EC022242092E0032092E103BE
:101910000E945B1DA09014042A2C3324822D992749
:101920008050994F2C01420C531C5982488220EE62
:1019300033E002E00E945C1D809114048F5F80936D
:10194000140480911404843BF0F2222420922E048B
:1019500020922B04332430922D0420922C04809169
:1019600038038F7D80933803309838988D7F80932B
:1019700038032092360420923704209232042092B9
:1019800031042092300488E78093330420925F046E
:1019900030925D0420925C0488E880931504809165
:1019A00038038064809338038F7780933803846092
:1019B00080933803877F80933803809137038B7F30
:1019C00080933703877F809337038F7D809337031E
:1019D00080E98AB9809136038E7F809336038091A7
:1019E00035038D7F80933503809136038D7F8093FF
:1019F00036038F7D809336038F7E80933603877FF7
:101A0000809336038B7F8093360380E981B9949865
:101A100020926B0381B5886181BD8FE081BD789490
:101A20000C94621BA89580913803817009F47EC1E3
:101A3000809137039927959587959595879581701E
:101A400090708030890709F471C1809138038E7FCE
:101A50008093380385E020903004821560F4209054
:101A60003304222041F48093300480E090E290938C
:101A7000B4038093B3038FEF90E02090B3033090D2
:101A8000B4038215930540F5AA9AAB9830923403BB
:101A90002092330320903403209214040AC08091D2
:101AA0002B048F5F80932B04863018F02224209221
:101AB0002B0410912B0401E00E94951F2090140428
:101AC000202269F3A0902B048A2D8F5F80932B0432
:101AD0000A2D0E942F052AC12090B3033090B40331
:101AE000222019F4332009F4A6C0AA98AB9A3092A8
:101AF000340320923303209214040AC080912B04F3
:101B00008F5F80932B04863018F0222420922B04C0
:101B100010912B0401E00E94951F209014042022B4
:101B200069F382E020902B04821558F48091B5036C
:101B30009091B6038030E0E89E0718F085E080932E
:101B40002B04A0902B048A2D8F5F80932B040A2DE9
:101B50000E94600580912E038F5F80932E03843056
:101B600069F48091B5039091B6038F3FEFE79E072C
:101B700028F480912E038F5F80932E038AE02090BB
:101B80002E03821518F481E080932E03A0902E037B
:101B9000BB24C5018130E0E09E0729F18230E0E0FE
:101BA0009E0729F18330E0E09E0729F18430E0E0D0
:101BB0009E0729F18530E0E09E0729F18630E0E0BC
:101BC0009E0729F18730E0E09E0729F18830E0E0A8
:101BD0009E0729F18930E0E09E0729F18A30E0E094
:101BE0009E0729F1A3C001E00E947D039FC001E090
:101BF0000E94A3039BC001E00E94C50397C001E0BF
:101C00000E94EB0393C001E00E9411048FC001E029
:101C10000E9435048BC001E00E947C0487C001E073
:101C20000E94A10483C001E00E94DF047FC001E0A4
:101C30000E9418057BC0AA9AAB9A80912E038F5FF1
:101C4000A82EA0922E0384E08A1518F42224209254
:101C50002E03A0902E03BB24AA2011F4BB2091F0E8
:101C6000C5018130E0E09E07A1F08230E0E09E07F0
:101C700019F18330E0E09E0731F18430E0E09E0707
:101C800049F154C000270E947D0301E00E94A30394
:101C90004DC000270E94C5038091B5039091B60303
:101CA0008F3FEFE79E0720F401E00E949D053EC0B4
:101CB00001E00E94EB033AC000270E94110401E0FA
:101CC0000E94350433C000270E947C0401E00E947A
:101CD000A1042CC027E030E00091360311270E94B8
:101CE0006D1EC8018170907080308907C9F021E0B5
:101CF00009E00E94261E2090170425FE08C080914E
:101D000036038068809336030E9482050CC0809160
:101D1000360380688093360300270E94DF0403C0E7
:101D200000270E94DF0401E00E941805809138031B
:101D3000992795958795817090708030890709F46F
:101D400036C4159B34C4A0909B03BB24C5018130CD
:101D5000E0E09E0709F433C08230E0E09E0709F41A
:101D60006FC08330E0E09E0709F42DC18430E0E0CD
:101D70009E0709F488C18530E0E09E0709F4E3C1BD
:101D80008630E0E09E0709F43EC28730E0E09E071F
:101D900009F493C28930E0E09E0709F4CFC28B308A
:101DA000E0E09E0709F40CC38C30E0E09E0709F4E4
:101DB0004CC38D30E0E09E0709F49FC3F6C320902A
:101DC0003604222039F585E08093410388E0809332
:101DD000420380916A038F778093430381E080936D
:101DE000440388E0809345038093460304E610E0B3
:101DF0000E94661BA0903604BB248A2D8F5F8093BF
:101E0000360481E493E0EA2DFF27E80FF91F2080D4
:101E100023B8CDC380913604863078F481E493E012
:101E2000E0913604FF27E80FF91F208023B8809146
:101E300036048F5F80933604BAC30E947F1CB7C3F9
:101E400020903604222009F0A9C085E08093410348
:101E500088E08093420382E0809343038CE1809387
:101E6000440320903D042092450320903F0420929B
:101E7000460380913E048F70829520904004282A6A
:101E8000209247032090410420924803209043046D
:101E9000209249032090440420924A032090450454
:101EA00020924B032090460420924C03209047043C
:101EB00020924D032090490420924E0320904A0422
:101EC00020924F0320904B04209250032090510405
:101ED00020925103209052042092520320915404E6
:101EE000332700E011E00E94301F20905304332478
:101EF000200E311E2AE030E081010E94781E0093FE
:101F000053032090550420925403209057042092AC
:101F10005503209069032092560320906A03209273
:101F2000570320906D032092580320906E03209257
:101F3000590320906F0320925A032090700320923F
:101F40005B032090710320925C0320907303209226
:101F50005D032090740320925E032090750320920D
:101F60005F0320907603209260030E943F07A02E1B
:101F7000A092610304E610E00E94661BA090360464
:101F8000BB248A2D8F5F8093360481E493E0EA2D91
:101F9000FF27E80FF91F208023B809C3809136047A
:101FA000813270F4A82EBB248F5F8093360481E4C5
:101FB00093E0EA2DFF27E80FF91F208023B8F7C22E
:101FC0000E947F1CF4C220903604222009F042C0F7
:101FD00085E08093410388E08093420384E8809306
:101FE000430388E18093440322242092140415C003
:101FF000A090140489E693E0EA2DFF27E80FF91F6B
:10200000208085E493E0EA2DFF27E80FF91F208266
:10201000809114048F5F809314048091140488319C
:1020200038F30E943F07A02EA0925D0304E610E063
:102030000E94661BA0903604BB248A2D8F5F80937C
:10204000360481E493E0EA2DFF27E80FF91F208092
:1020500023B8ADC2809136048D3170F4A82EBB2414
:102060008F5F8093360481E493E0EA2DFF27E80F29
:10207000F91F208023B89BC22224209236048CE0D2
:1020800080939B0394C220903604222009F042C022
:1020900085E08093410388E08093420388E8809341
:1020A00043038CE18093440322242092140415C03E
:1020B000A090140489E693E0EA2DFF27E80FF91FAA
:1020C000208085E493E0EA2DFF27E80FF91F2082A6
:1020D000809114048F5F80931404809114048C31D8
:1020E00038F30E943F07A02EA092610304E610E09F
:1020F0000E94661BA0903604BB248A2D8F5F8093BC
:10210000360481E493E0EA2DFF27E80FF91F2080D1
:1021100023B84DC280913604813270F4A82EBB24BE
:102120008F5F8093360481E493E0EA2DFF27E80F68
:10213000F91F208023B83BC22224209236048BE072
:1021400080939B0334C220903604222009F042C0C1
:1021500085E08093410388E08093420380E9809387
:10216000430388E18093440322242092140415C081
:10217000A090140489E693E0EA2DFF27E80FF91FE9
:10218000208085E493E0EA2DFF27E80FF91F2082E5
:10219000809114048F5F809314048091140488311B
:1021A00038F30E943F07A02EA0925D0304E610E0E2
:1021B0000E94661BA0903604BB248A2D8F5F8093FB
:1021C000360481E493E0EA2DFF27E80FF91F208011
:1021D00023B8EDC1809136048D3170F4A82EBB2454
:1021E0008F5F8093360481E493E0EA2DFF27E80FA8
:1021F000F91F208023B8DBC12224209236048DE011
:1022000080939B03D4C120903604222009F03FC064
:1022100085E08093410388E08093420380916A03C4
:102220008F778093430386E0809344032090690373
:102230002092450320906A032092460320906B036E
:102240002092470320906C032092480320906D0356
:102250002092490320906E0320924A030E943F0778
:10226000A02EA0924B0304E610E00E94661BA090F3
:102270003604BB248A2D8F5F8093360481E493E07B
:10228000EA2DFF27E80FF91F208023B890C1809125
:1022900036048B3078F481E493E0E0913604FF2734
:1022A000E80FF91F208023B8809136048F5F809358
:1022B00036047DC10E947F1C7AC120903604222002
:1022C00039F585E08093410388E080934203809153
:1022D0006A038F778093430381E08093440387E010
:1022E000809345038093460304E610E00E94661B3A
:1022F000A0903604BB248A2D8F5F8093360481E43E
:1023000093E0EA2DFF27E80FF91F208023B84FC183
:1023100080913604863078F481E493E0E0913604CD
:10232000FF27E80FF91F208023B8809136048F5FC4
:10233000809336043CC10E947F1C39C12090360432
:10234000222049F585E08093410388E08093420391
:1023500089E08093430382E08093440320905704F4
:102360002092450320905804209246030E943F0784
:10237000A02EA0924703A0903604BB248A2D8F5F25
:102380008093360481E493E0EA2DFF27E80FF91FDC
:10239000208023B80CC180913604873070F4A82EB9
:1023A000BB248F5F8093360481E493E0EA2DFF27FE
:1023B000E80FF91F208023B8FAC00E947F1CF7C0E5
:1023C00020903604222061F585E08093410388E067
:1023D000809342038093430383E0809344032090DF
:1023E0008503209245032090860320924603209087
:1023F0008703209247030E943F07A02EA092480324
:10240000A0903604BB248A2D8F5F8093360481E42C
:1024100093E0EA2DFF27E80FF91F208023B8C7C0FB
:1024200080913604883070F4A82EBB248F5F80938F
:10243000360481E493E0EA2DFF27E80FF91F20809E
:1024400023B8B5C00E947F1CB2C020903604222061
:1024500009F03EC085E08093410388E08093420309
:1024600084E08093430388E18093440322242092F4
:10247000140415C0A090140481E893E0EA2DFF270E
:10248000E80FF91F208085E493E0EA2DFF27E80F8D
:10249000F91F2082809114048F5F8093140480912F
:1024A0001404883138F30E943F07A02EA0925D03E8
:1024B000A0903604BB248A2D8F5F8093360481E47C
:1024C00093E0EA2DFF27E80FF91F208023B86FC0A3
:1024D000809136048D3170F4A82EBB248F5F8093D9
:1024E000360481E493E0EA2DFF27E80FF91F2080EE
:1024F00023B85DC00E947F1C5AC020903604222061
:1025000009F03EC085E08093410388E08093420358
:1025100080E18093430388E1809344032224209246
:10252000140415C0A090140481E893E0EA2DFF275D
:10253000E80FF91F208085E493E0EA2DFF27E80FDC
:10254000F91F2082809114048F5F8093140480917E
:102550001404883138F30E943F07A02EA0925D0337
:10256000A0903604BB248A2D8F5F8093360481E4CB
:1025700093E0EA2DFF27E80FF91F208023B817C04A
:10258000809136048D3170F4A82EBB248F5F809328
:10259000360481E493E0EA2DFF27E80FF91F20803D
:1025A00023B805C00E947F1C02C00E947F1C80913E
:1025B000380399279595879595958795959587954E
:1025C000817090708030890709F43FC222242092E4
:1025D0005B0482E08093140412C089E394E0E091EC
:1025E0001404FF27E80FF91F208030905B04320CA1
:1025F00030925B04809114048F5F80931404809167
:102600001404803250F38091370384608093370341
:102610002224209230042090590430905B0432141C
:1026200009F00BC220903B042092330320903C041D
:102630002092340320903303309034033092D4033B
:102640002092D30320903D042092330320903E0437
:102650002092340320903303309034033092D2031D
:102660002092D10320903F04209233032090400415
:102670002092340320903303309034033092D003FF
:102680002092CF03209041042092330320904204F3
:102690002092340320903303309034033092CE03E1
:1026A0002092CD03209043042092330320904404D1
:1026B0002092340320903303309034033092CC03C3
:1026C0002092CB03209045042092330320904604AF
:1026D0002092340320903303309034033092CA03A5
:1026E0002092C9032090470420923303209048048D
:1026F0002092340320903303309034033092C60389
:102700002092C503209049042092330320904A046C
:102710002092340320903303309034033092C80366
:102720002092C70320904B042092330320904C0446
:102730002092340320903303309034033092C4034A
:102740002092C30320904D042092330320904E0426
:102750002092340320903303309034033092C2032C
:102760002092C10320904F04209233032090500404
:102770002092340320903303309034033092C0030E
:102780002092BF03209053042092330320905404DE
:102790002092340320903303309034033092B803F6
:1027A0002092B70380E820905504821538F4809178
:1027B0003703806280933703A99806C0809137035E
:1027C0008F7D80933703A99A20905504209233037C
:1027D0002090560420923403209033033090340329
:1027E0003092B6032092B5032090550426FE09C00E
:1027F0008091B5039091B60390689093B60380934F
:10280000B503809157048F718093330380915804EE
:102810008F718093340320903303309034033092CF
:10282000B4032092B303A090B303B090B4032090FC
:102830002C0430902D042A143B0471F0AA2011F4CA
:10284000BB2051F0809138038062809338031501DA
:1028500030922D0420922C042090510420923303B6
:1028600020905204209234032AE030E00091330398
:10287000109134030E94941E1093BE030093BD0375
:1028800021E006EF15E00E94DF1D2090E00320927A
:1028900011042090BD033090BE0330923403209287
:1028A00033032092E003209034032092E1030E943E
:1028B0005B1D209011043324822D99278050994F5D
:1028C0002C01420C531C5982488220EE33E002E076
:1028D0000E945C1D809111048F5F8093E0030E9431
:1028E0005B1D86EF95E09983888320EE33E001E05D
:1028F0000E945C1D80913603817009F46AC080914A
:1029000036038E7F809336038091350381608093F8
:10291000350386E080935E0488E08AB92224209201
:10292000360481EF8093690380936A0388E0809383
:102930006B032090D60320926C032090D703209243
:102940006D032090D80320926E032090D90320922B
:102950006F032090DA03209270032090DB03209213
:1029600071032090DC03209272032090DD032092FB
:1029700073032090D7033090D603320C2090D803F5
:10298000320C2090D903320C2090DA03320C2090C4
:10299000DB03320C2090DC03320C2090DD03320C80
:1029A0003092740310C05D9B0EC089E693E0E09105
:1029B0003604FF27E80FF91F20802CB880913604D9
:1029C0008F5F80933604809136048C3060F380E909
:1029D0008AB980913503817081F120905E042220B4
:1029E00061F1822D815080935E04882339F48091B7
:1029F00035038E7F809335030E947F1C80913A04BB
:102A0000813711F08135C9F480913A04813731F46E
:102A10008091350384608093350305C08091350330
:102A20008B7F809335030E947F1C809135038E7FBE
:102A300080933503826080933503809138038460EE
:102A400080933803877F80933803809138039927D8
:102A5000959587959595879595958795959587955E
:102A6000817090708030890709F4FBC10E942D07A6
:102A7000809138038F7E8093380380E08093B90380
:102A80008093BA038093BB038093BC0321E006EFDD
:102A900015E00E94DF1D2090E0032092110484EBDA
:102AA000821510F48093110422242092140434C05F
:102AB00022E0A09014042A2C3324022D1127005068
:102AC000194F020D131D0E94DF1D2090E00320927C
:102AD00033032090E103209234032090330330909D
:102AE0003403442455248090BB039090BC03609031
:102AF000B9037090BA03620C731C841C951C70920D
:102B0000BA036092B9039092BC038092BB03809198
:102B100014048F5F80931404209011043324409098
:102B200014045524241435041CF644EB50E060E0F2
:102B300070E02091BB033091BC030091B903109168
:102B4000BA037A936A935A934A930E94AE1E1093E3
:102B5000BE030093BD0322242092E0030E945B1D6C
:102B600086EF95E09983888320EE33E001E00E94B0
:102B70005C1D2090BD033090BE034090A203509096
:102B8000A303420C531C5092A3034092A203409013
:102B9000A0035090A103420C531C5092A1034092F9
:102BA000A00328EE33E00091A2031091A3030E943A
:102BB000941E00931404202E002309F470C03324C3
:102BC0004090A4035090A503420C531C5092A503BF
:102BD0004092A403222D332708EE13E00E94301FF9
:102BE0002090A2033090A303201A310A3092A3034D
:102BF0002092A203209014043090AE03320C309245
:102C0000AE031AE0032D0E941A1F002309F447C0E7
:102C10008091AE038A508093AE0341E050E060E0C3
:102C200070E04090B1035090B2032090AF03309019
:102C3000B003240E351E461E571E3092B00320925C
:102C4000AF035092B2034092B10340EE53E964E007
:102C500070E0241635064606570648F080E080935B
:102C6000AF038093B0038093B1038093B20341E03C
:102C700050E060E070E040909E0350909F032090F1
:102C80009C0330909D03240E351E461E571E309225
:102C90009D0320929C0350929F0340929E0380913B
:102CA000A7039091A80301969093A8038093A7038C
:102CB0008091A9038F5F8093A90341E050E060E019
:102CC00070E04090AC035090AD032090AA03309088
:102CD000AB03240E351E461E571E3092AB032092C6
:102CE000AA035092AD034092AC0389E02090A9035F
:102CF000821518F422242092A9034090B103509029
:102D0000B2032090AF033090B00330923003209292
:102D10002F0350923203409231032092E00320901F
:102D200030032092E103209031032092E2032090AF
:102D300032032092E3032090AE032092E4034090FC
:102D4000AC035090AD032090AA033090AB033092B7
:102D5000300320922F03509232034092310320928D
:102D6000E503209030032092E60320903103209267
:102D7000E703209032032092E8032090A7033090CD
:102D8000A80330923403209233032092E903209069
:102D900034032092EA032090A4033090A5033092DC
:102DA0003403209233032092EB03209034032092CB
:102DB000EC032090A2033090A303309234032092BE
:102DC00033032092ED03209034032092EE032090F1
:102DD000A0033090A1033092340320923303209259
:102DE000EF03209034032092F0032090A903209257
:102DF000F10340909E0350909F0320909C033090DD
:102E00009D033092300320922F0350923203409260
:102E100031032092F203209030032092F30320909C
:102E200031032092F403209032032092F50326E030
:102E300003E00E94261EF8940E945B1D80EE95E040
:102E40009983888320EE33E006E10E945C1D2224F2
:102E500033243982288227E134E006E00E945C1D99
:102E600078948091370399279595879595958795BF
:102E7000817090708030890709F4CDC00E942D07C1
:102E800080912F048F5F80932F0481E020902F0486
:102E9000821528F4809136038D7F8093360326E0D7
:102EA00003E00E94261E2090170420922004209008
:102EB00018042092230420901A04209226042090C3
:102EC0001B042092280420901C04209229040091C5
:102ED00020040E940107A02E2090A6033A2C320C59
:102EE00030921404A09015048A2D883821F0232CE8
:102EF000821509F490C0209014042092150416E065
:102F0000022D0E94181F002329F48091380380614C
:102F10008093380380912304833259F480912004F4
:102F2000893539F4009126040E940107A02EA09251
:102F3000240420902004222009F06DC00091230475
:102F40000E940107A02EA0922104009126040E9455
:102F50000107A02EA09225040E945D062090210466
:102F6000222009F052C020902404209225040E94BF
:102F70009F060E945D06222433243092A1032092F2
:102F8000A0033092A5032092A4033092A8032092BC
:102F9000A703009126040E940107A02EA0922504F9
:102FA00022242092210407C00E945D068091210402
:102FB0008F5F80932104809121048831A8F322241B
:102FC00020922104809126048130F9F40091280494
:102FD0000E940107A02EA0922704013021F48CE06A
:102FE0008093270405C08091270481508093270493
:102FF000009127040E94C30680E080939C03809385
:103000009D0380939E0380939F0322243324309258
:10301000A1032092A003A090380327E030E00A2DFE
:1030200011270E946D1EC801817090708030890741
:1030300009F4BFC28A2D9927959587958170907064
:103040001C0120943094222019F4332009F4B1C2D9
:10305000809138038F778093380380916A038A3A8E
:1030600009F492C280916A03823C39F585E0209090
:1030700033048215D8F420906C032092E003209052
:103080006D032092E10320906E032092E2030E94E0
:103090005B1D86E09FE19983888320EE33E003E0A7
:1030A0000E945C1D81E080939B0303C087E08093B6
:1030B0009B0382E480936B0367C280916A03813C27
:1030C00059F585E0209033048215F8F420906C03C4
:1030D0002092E00320906D032092E10320906E0384
:1030E0002092E20320906F032092E3030E945B1D75
:1030F00089E09FE19983888320EE33E004E00E9419
:103100005C1D81E080939B0303C087E080939B0359
:1031100081E480936B0338C280916A03803C09F09C
:1031200056C0809135039927959587958170907049
:1031300080308907D1F0809135038D7F80933503EE
:103140009927959587959595879581709070803092
:10315000890721F081E080939B0303C087E080937F
:103160009B0380E480936B030FC2809136038170D0
:10317000813049F18091360381608093360320903D
:103180006C032092D60320906D032092D7032090E9
:103190006E032092D80320906F032092D9032090D1
:1031A00070032092DA03209071032092DB032090B9
:1031B00072032092DC03209073032092DD0322240B
:1031C00020929B03E1C1222420929B03DDC18091C8
:1031D0006A03813809F03BC022242092140415C0F0
:1031E000A09014048CE693E0EA2DFF27E80FF91F66
:1031F000208087E194E0EA2DFF27E80FF91F208265
:10320000809114048F5F809314048091140487309C
:1032100038F327E002E00E94B01D209018042092AD
:103220002004209019042092230420901B04209253
:10323000260420901C042092280420901D04209233
:10324000290481E080936B0380939B039DC180914F
:103250006A03823009F06AC02090A4033090A5036D
:10326000442455243092300320922F03509232038D
:1032700040923103209269032090300320926A0328
:103280002090310320926B032090320320926C0334
:103290004090B1035090B2032090AF033090B00340
:1032A0003092300320922F03509232034092310328
:1032B00020926D032090300320926E032090310302
:1032C00020926F0320903203209270032090A70376
:1032D0003090A8033092340320923303209271037C
:1032E00020903403209272034090AC035090AD03C1
:1032F0002090AA033090AB033092300320922F032A
:103300005092320340923103209273032090300395
:103310002092740320903103209275032090320391
:103320002092760382E080939B032EC180916A03F2
:10333000843009F063C020906C0320929A03022D20
:103340000E940107A02E80E38A9DC001C097909340
:1033500013048093120420E38C010E94DF1D2224B9
:103360002092140415C0A090140480EE93E0EA2D7E
:10337000FF27E80FF91F208089E693E0EA2DFF2759
:10338000E80FF91F2082809114048F5F809314044A
:1033900080911404803338F320909A0330902604EF
:1033A000321441F52090A0033090A10330923403F1
:1033B00020923303009123040E940107A02E89E686
:1033C00093E0EA2DFF27EE0FFF1FE80FF91F209073
:1033D00033032082009123040E940107A02E8AE675
:1033E00093E0EA2DFF27EE0FFF1FE80FF91F209053
:1033F0003403208283E080939B03C6C080916A03DC
:10340000883041F50E949F062FE100E016E00E94FF
:10341000DF1D22242092140415C0A090140480EE15
:1034200093E0EA2DFF27E80FF91F208089E693E05B
:10343000EA2DFF27E80FF91F2082809114048F5F87
:1034400080931404809114048F3138F384E08093C6
:103450009B039AC080916A03803179F5009128041A
:103460000E940107A02EA09227040E94C30620E319
:1034700000E916E00E94DF1D22242092140415C0EA
:10348000A090140480EE93E0EA2DFF27E80FF91FC7
:10349000208089E693E0EA2DFF27E80FF91F2082BC
:1034A000809114048F5F80931404809114048033FE
:1034B00038F385E080939B0367C080916A03803274
:1034C00009F04EC020906C032092330320906D03CE
:1034D00020923403209133033091340305E010E04F
:1034E0000E94301FC8018052964F909334038093FE
:1034F000330388E69DE12090330330903403821536
:10350000930530F480EE99E0909334038093330375
:1035100026E000913303109134030E94DF1D222422
:103520002092140415C0A090140480EE93E0EA2DBC
:10353000FF27E80FF91F208089E693E0EA2DFF2797
:10354000E80FF91F2082809114048F5F8093140488
:1035500080911404863038F386E080939B0314C076
:1035600080916A038F3F21F489E080939B030CC014
:1035700080916A03833441F48091360382608093A2
:103580003603222420929B0320909B03222061F08B
:10359000222420923604809138038260809338037D
:1035A00088E081B9949A05C0809138038064809343
:1035B000380325E030E00091380311270E946D1E8A
:1035C000C801817090708030890709F464C08091CF
:1035D00038038F7D8093380322E007EF15E00E94C7
:1035E000DF1D2090E003209233032090E10320921E
:1035F0003403209020042092E003209023042092A2
:10360000E103209026042092E20320902C043090C5
:103610002D04232C33242092E30320902C0430909B
:103620002D042092E4030E945B1D20903303309010
:1036300034033982288220EE33E005E00E945C1DCD
:1036400080913303909134038836EDE19E0738F082
:1036500080EE99E0909334038093330309C0809106
:10366000330390913403059690933403809333038E
:10367000209033032092E003209034032092E10352
:103680000E945B1D87EF95E09983888320EE33E0ED
:1036900002E00E945C1D80913703992795958795DC
:1036A0009595879595958795959587958170907057
:1036B0008030890739F0809137038F7E80933703FC
:1036C0000E947F1C0C94120D229608954A935A93DF
:1036D00009C04427552702C04F5F5F4F403AE0E0E2
:1036E0005E07D0F3180101501040222091F73320DB
:1036F00081F75991499108952A928A939A93EA936E
:10370000FA932FB62A9220903803822D9927959507
:103710008795959587958170907080308907F9F02D
:10372000822D992795958795959587959595879558
:10373000817090708030890791F42CB02092390408
:10374000822D813F09F058C0809138038B7F809390
:10375000380381E080933804809332044DC0809117
:10376000380399279595879595958795959587958C
:10377000817090708030890709F03EC080913804D4
:103780008130B1F42CB020923A0482E08093380466
:1037900080913904813F81F180913803877F809344
:1037A000380384608093380322242092320424C09A
:1037B00080913804813278F489E394E0E091380410
:1037C000FF27E80FF91F2CB02082809138048F5F0B
:1037D0008093380411C08091380388608093380347
:1037E00089E394E0E0913804FF27E80FF91F2CB03B
:1037F000208222242092320429902FBEF991E9914F
:1038000099918991299018958898899A919A8FE52C
:1038100089B9222420BC2BB82AB886E880BD089537
:103820002A920A931A932A933A938A939A93EA9341
:10383000FA932FB62A9226E030E000913803112740
:103840000E946D1EC8018170907080308907C9F098
:10385000809137048230A8F423B020926903822D2E
:103860008A3A09F034C0809138038F7B8093380303
:10387000809137048F5F8093370481E08093310417
:1038800026C080916B038C5F20903704281670F45B
:1038900088E693E0E22DFF27E80FF91F23B020828E
:1038A000809137048F5F8093370411C08091380373
:1038B00080688093380388E693E0E0913704FF271F
:1038C000E80FF91F23B0208222242092310429908E
:1038D0002FBEF991E9919991899139912991199185
:1038E000099129901895BA98BB9A8FE580B922243E
:1038F0002CBE22B880E881B986E88CBF08950027E5
:10390000112704C0000000000F5F1F4F0038E6E0E1
:103910001E07C0F3222420926B03809138038D7F11
:103920008093380388E081B9949A80E482B980E971
:1039300081B994982092370420929B038091380398
:1039400080648093380308952227332700271127A6
:10395000E6D021E030E001E010E0E1D0222733277B
:1039600009E010E0DCD0222733270BE010E0D7C0BD
:103970008F9A8E9A969808950027112703C0000009
:103980000F5F1F4F0A30E0E01E07C8F308954A9307
:103990005A930BC04427552703C000004F5F5F4F69
:1039A0004A30E0E05E07C8F30A9580E0801790F3A4
:1039B0005991499108954A935A930AC0442755272B
:1039C00002C04F5F5F4F4032E3E05E07D0F30A95DD
:1039D00080E0801798F35991499108958F9A05E0F6
:1039E000D6DF979AC9DF969AC7DF979802E0E3DFA0
:1039F0009698C2DF01E0DFCF969ABEDF8F9A05E08E
:103A0000C6DF9798B9DF979AB7CF8F9A9798B4DFA8
:103A1000969AB2DF9698B0DF979A08958F9A979A00
:103A2000ABDF969AA9DF9698A7CF4A938F98A4DF29
:103A3000969A05E0ACDF40B340789EDF969805E0AB
:103A4000A6DF042F499108950E945E1F602F8F9A70
:103A500048E011C0862F8078A82E803811F4979AFC
:103A600001C0979889DF969A05E091DF969805E066
:103A70008EDF660F4A95442369F70C94651F0E94F8
:103A80005E1F44278F9868E011C0969A05E07FDF9B
:103A9000440F80B38078A82E803811F4416000C0B4
:103AA00005E075DF969805E072DF6A95662369F791
:103AB000042F0C94651F08950E947A1FA901A02E5F
:103AC000C884D9848BDF00EABFDFAFDF003811F490
:103AD00001E023C08601012F1127B6DFA6DF0038E1
:103AE00011F401E01AC00C2DAFDF9FDF602F00380A
:103AF00071F401E012C0FA010081A6DF96DF602FA9
:103B0000003811F401E009C04F5F5F4FAA94AA206A
:103B100091F772DF01E04FDF00270C94831F0E94B2
:103B20006C1FA22EC02E5ADF00ED8EDF7EDF003824
:103B300011F401E013C00C2D87DF77DF003811F49A
:103B400001E00CC00A2D80DF70DF402F003811F437
:103B500001E004C051DF01E02EDF00270C94731F49
:103B60000E944B1FC22EE02EAA2422E00027D7DF9E
:103B700035DF00ED69DF59DF003811F401E01DC0C9
:103B80000E2D62DF52DF003891F401E016C087E1AC
:103B900094E0EA2DFF27E80FF91F008155DF45DF8C
:103BA000402F003811F401E008C0A394CA94CC203F
:103BB00071F722DF03E0EBDE00270C94401F0E9428
:103BC0007A1F422F5801CC2409DF00EA3DDF2DDFA8
:103BD000003811F401E038C0CFDE8501012F112734
:103BE00033DF23DF003811F401E02EC0C5DE0A2DDB
:103BF0002BDF1BDF602F003811F401E025C0EEDE63
:103C000001EA22DF12DF602F003871F401E01CC0EE
:103C100036DFA02E80EE93E0EC2DFF27E80FF91F92
:103C2000A082F3DEC3944A95413091F728DFA02E9D
:103C300080EE93E0EC2DFF27E80FF91FA082EEDE67
:103C4000DBDE03E0A4DE00270C94831F0E947A1FB2
:103C5000422FA02ECC2421E0002761DFBFDE00ED43
:103C6000F3DEE3DE003811F401E030C085DE0A2D1A
:103C7000EBDEDBDE003811F401E028C0AFDE01ED41
:103C8000E3DED3DE602F003871F401E01FC0F7DE01
:103C9000A02E87E194E0EC2DFF27E80FF91FA0820A
:103CA000B4DEC3944A95413091F7E9DEA02E87E156
:103CB00094E0EC2DFF27E80FF91FA082AFDE9CDE19
:103CC00003E065DE222700272ADF00270C94831FEC
:103CD0003A932A931A930A930895222321F0159573
:103CE00007952A95FACF08956894DA92D12E04C0E8
:103CF000E894DA92D12ED32617FF04C010950095D0
:103D00000F5F1F4F37FF04C0309520952F5F3F4F47
:103D10000E94951ED7FE04C0109500950F5F1F4F9F
:103D2000D9900895689401C0E894EA92FA928A932F
:103D3000EE24FF2480E1000F111FEE1CFF1CE21691
:103D4000F30618F0E21AF30A03958A95A1F716F420
:103D50000E2D1F2D8991F990E9900895E89401C0E6
:103D6000689430D0CC2409C0E89401C068942AD06B
:103D700037FD0E948C1FB7FD52D0772488249924E8
:103D8000AA24BB2442D0C1F045D0B1F0E8E2000F34
:103D9000111F221F331F771C881C991CAA1CBB1CD7
:103DA00088169906AA06BB0628F0881A990AAA0A54
:103DB000BB0A0395EA9559F726F4082D192D2A2DEB
:103DC0003B2D13C07A928A929A92AA92BA92CA9280
:103DD000EA938A939A93AA93BA938B859C85AD852F
:103DE000BE85C32E0EF0CB260895C7FC0E948C1F03
:103DF000B991A99199918991E991C990B990A990A6
:103E000099908990799024960895E02FE12BE22BE8
:103E1000E32B0895E82FE92BEA2BEB2B08958095EF
:103E20009095A095B0958F5F9F4FAF4FBF4F08956E
:103E3000689401C0E8942A93FA92EA92FF24EE244F
:103E400020E1000FFF1CEE1CE11610F0E11A0395B3
:103E50002A95B9F70EF40E2DE990F990299108955D
:103E60000A921A928A939A93029FC001129F900D10
:103E7000039F900D8C019991899119900990089553
:103E8000A990B990C990D990E990F9904991599128
:103E900008957A936A935A934A93FA92EA92DA923D
:103EA000CA92BA92AA9208957A936A935A934A93BD
:103EB0000895499159916991799108957A936A93F6
:103EC0005A934A93BA92AA920895A990B9904991A7
:103ED00059916991799108955A934A93DA92CA92C5
:103EE000BA92AA920895A990B990C990D99049918F
:103EF000599108957A936A935A934A93DA92CA929F
:103F0000BA92AA920895A990B990C990D99049916E
:103F10005991699179910895009510952095309562
:103F20000F5F1F4F2F4F3F4F0895112319F0000FC0
:103F30001A95FBCF0895FFFFFFFFFFFFFFFFFFFF75
:103F4000FFFFFFFFFFFFFFFFFFFFFFFFFFFFFFFF81
:103F5000FFFFFFFFFFFFFFFFFFFFFFFFFFFFFFFF71
:103F6000FFFFFFFFFFFFFFFFFFFFFFFFFFFFFFFF61
:103F7000FFFFFFFFFFFFFFFFFFFFFFFFFFFFFFFF51
:103F8000FFFFFFFFFFFFFFFFFFFFFFFFFFFFFFFF41
:103F9000FFFFFFFFFFFFFFFFFFFFFFFFFFFFFFFF31
:103FA000FFFFFFFFFFFFFFFFFFFFFFFFFFFFFFFF21
:103FB000FFFFFFFFFFFFFFFFFFFFFFFFFFFFFFFF11
:103FC000FFFFFFFFFFFFFFFFFFFFFFFFFFFFFFFF01
:103FD000FFFFFFFFFFFFFFFFFFFFFFFFFFFFFFFFF1
:103FE000FFFFFFFFFFFFFFFFFFFFFFFFFFFFFFFFE1
:103FF000FFFFFFFFFFFFFFFFFFFFFFFFFFFFFFFFD1
:00000001FF
